:1000000012C0C8C72BC02AC029C028C027C026C01C
:1000100025C065C923C022C021C020C01FC01EC08A
:100020001DC01CC01BC011241FBECFE5D4E0DEBF25
:10003000CDBF11E0A0E6B0E0EAE7F5E102C005902F
:100040000D92A837B107D9F713E0A8E7B1E001C0D6
:100050001D92A434B107E1F7F5D38DCAD1CF482F53
:1000600090E820E030E0FB01E20FF31F892F8423AA
:10007000808396952F5F3F4F28303105A1F7089573
:10008000992787FD9095A92FB92FBC01CD0120ECB0
:100090003DE540E050E0D9D92FEF3FE740E050E0A8
:1000A000F3D9822F08956F927F928F929F92AF9291
:1000B000BF92CF92DF92EF92FF920F931F937C013A
:1000C0008B01FC0186818071FB018183F7018681B0
:1000D0008870FB018583F70186818078FB01818729
:1000E000F70186818170FB018587F7018681807227
:1000F000FB01818BF70186818074FB01858B38E1E0
:10010000632E712C660E771EF70183818058F301F0
:100110008183F70183818058FB01858F20E2822E45
:10012000912C860E971EF70182818058F4018183FD
:10013000F70182818058FB0185A3F70187818170D7
:10014000FB0181A7F70187818270FB0185A7F70179
:1001500087818870FB0181ABF70187818470FB0187
:1001600085AB98E3A92EB12CA60EB71EF7018081AE
:10017000805886DFF50181838CE3C82ED12CC00E18
:10018000D11EF701818180587BDFF6018183005CFD
:100190001F4FF70186818470F80181830C5F1F4F28
:1001A000F70186818270F80181830C5F1F4FF60191
:1001B0008181F80181830C5F1F4FF6018181F80175
:1001C00081830C5F1F4FF5018181F80181830C5FF2
:1001D0001F4FF5018181F80181830C5F1F4FF701EB
:1001E00084818058F80181830C5F1F4FF70185815E
:1001F0008058F80181830C5F1F4FF4018181F80161
:1002000081830C5F1F4FF3018181F80181831F916E
:100210000F91FF90EF90DF90CF90BF90AF909F90A5
:100220008F907F906F900895CF93DF93C0E0DAEFC7
:10023000CE010197F1F7E091FA01F091FB010484FE
:10024000F585E02D0995E091FA01F091FB01068416
:10025000F785E02D0995882359F3E091FA01F09193
:10026000FB010088F189E02D8CEF91E009958CEF7E
:1002700091E06EEA70E017DF20E030E08091AF009F
:10028000882311F021E030E08091B30081112260D9
:100290008091EF00811124608091F300811128602A
:1002A0008091B700811120618091BF00811120628F
:1002B0008091C300811120648091D7008111206852
:1002C0008091DB00811131608091DF00811132600B
:1002D0008091E300811134608091BB00811138600E
:1002E000E0917A01F0917B01E227F32741E050E0B1
:1002F00060E070E0CA018E239F23892B69F0CA0158
:1003000082239323892B41F030937B0120937A0140
:10031000CA01DF91CF910895440F551F6F5F7F4F42
:100320006C30710539F730937B0120937A0180CFCF
:10033000DF92EF92FF920F931F93CF93DF937B0196
:10034000D42E052F8032910519F0EB0110E80EC074
:10035000FB0180819181FFEF8F3F9F0709F451C01E
:100360000196FB019183808349C05EDF883091054F
:10037000D1F1893091054CF48230910561F18430DE
:10038000910569F1019789F723C08032910579F1D0
:10039000F8E080309F07A9F1409739F7103841F015
:1003A000188319828D2D902F9C01E90110E8DDCF73
:1003B000F70180819181FFEF8F3F9F0711F1019637
:1003C000F701918380838D2D902F9C01E901CDCF82
:1003D000110F110FCACF110F110F1F5FC6CF110FD1
:1003E000110F1E5FC2CF110F110F1D5FBECFCE15B3
:1003F000DF0539F0103811F01883198220E030E061
:1004000002C02FEF3FEFC901DF91CF911F910F91F4
:10041000FF90EF90DF900895CF93DF93DC01EB0125
:1004200020E011969C91119713968C911397981335
:1004300021E02883FD01349620E091818381981387
:1004400021E02983FD01389620E091818381981372
:1004500021E02A83FD013C9620E09181838198135D
:1004600021E02B83FD01B89620E0918183819813D0
:1004700021E02C83FD01BC9620E0918183819813BB
:1004800021E02D83FD01F09620E091818381981376
:1004900021E02E83FD01F49620E091818381981361
:1004A00021E02F8318861986FD01709620E0918146
:1004B0008381981321E02A87FD01749620E09181C1
:1004C0008381981321E02B87FD01789620E09181AC
:1004D0008381981321E02C87FD017C9620E0918197
:1004E0008381981321E02D87FD01B09620E0918152
:1004F0008381981321E02E87FD01B49620E091813D
:100500008381981321E02F87D9963C91D997DD9666
:100510002C91DD97FD01E05CFF4F9181838198175D
:1005200009F4922FFD01EC5BFF4F51818381581735
:1005300009F4592FFD01E85BFF4F918183819817E2
:1005400009F4932FFD01E45BFF4F4181838148173C
:1005500009F4492FFE01709690E89E01285E3F4FF6
:10056000892F842381939695E217F307C9F7252FE6
:10057000209590E8BE01605E7F4F892F8223819392
:100580009695E617F707C9F7DF91CF910895A4E094
:10059000B2E0E0E6F0E028E301900D922150E1F7AF
:1005A0009C012150304024303105C0F488E390E0B4
:1005B000289FF001299FF00D389FF00D1124EC5B6E
:1005C000FD4F80818F3F19F42FEF3FEF09C0A4E06A
:1005D000B2E088E301900D928150E1F720E030E035
:1005E000C90108959C01215030402430310598F410
:1005F00088E390E0289FF001299FF00D389FF00DCF
:100600001124EC5BFD4FA4E0B2E088E30D90019271
:100610008150E1F792D6089581E090E03ED604DE65
:1006200022E080309207D9F022E0813092073CF43A
:100630008038910571F08050914041F40DC024E064
:100640008030920779F08050984081F02FEF3FEF93
:1006500012C081E090E008C082E090E005C083E035
:1006600090E002C084E090E0BDDF03C080E090E055
:100670008EDF20E030E0C9010895DF92EF92FF9213
:100680000F931F93DF93CF9300D000D0CDB7DEB789
:100690008FEF9FEF9A8389839C838B83DFB6F894D7
:1006A000EDD585E090E0F9D500E01AEFE091FA0190
:1006B000F091FB010484F585E02D0995E091FA01A4
:1006C000F091FB010088F189E02D8CEF91E0099514
:1006D0008CEF91E06EEA70E0E6DC8091BB0088234D
:1006E00021F0C8010197F1F7E1CFB3E0EB2EF12C37
:1006F000EC0EFD1E8E010F5F1F4F96DD9C018032B8
:10070000910509F443C08132910594F48430910538
:1007100009F43CC08530910524F40197029768F7ED
:1007200035C08830910591F18031910531F72EC0A7
:1007300081E020303807D9F081E0213038073CF4DF
:1007400020343105F1F020383105B9F60DC084E0D0
:100750002030380791F088E02030380709F443C092
:100760002050324051F606C081E090E008C082E09F
:1007700090E005C083E090E002C084E090E007DFF5
:1007800001C04ADF8F5F9F4F71F51AC0C901B801E0
:10079000A701CEDD8F5F9F4F99F069817A818FEF3E
:1007A0006F3F780769F04B815C812FEF4F3F520715
:1007B00039F084E092E0CCD481E090E06ED59DCF1A
:1007C00083E090E06AD581E090E05BD588E59BE12D
:1007D00020E931E0F9013197F1F70197D9F780E08D
:1007E00090E04FD503C083E090E057D5DED5DFBE63
:1007F0000F900F900F900F90CF91DF911F910F915D
:10080000FF90EF90DF900895FC018585882391F09B
:100810008AD5882399F08091780190917901019689
:100820009093790180937801069744F026DF21E0C8
:1008300030E006C0109279011092780120E030E09B
:10084000C9010895C2D09093FB018093FA0111BAB7
:1008500082B38B6F82BB889A14BA8FEF85BB85B742
:10086000886085BF85B78B7F85BF8BB780648BBF62
:100870002EEA31E0C90160E070E040E250E04ED67F
:100880002EEC31E0C90160E070E040E250E046D675
:1008900095E09093EE011092EF0182E08093F001D9
:1008A0009093F1011092F2011092F3017894E6D442
:1008B0004CD5892B19F082E090E0EFD4809143026F
:1008C00090E065DE27D5E091FA01F091FB0102840A
:1008D000F385E02D0995909A88E893E120E931E0CD
:1008E000F9013197F1F70197D9F7E091FA01F09109
:1008F000FB010484F585E02D0995E091FA01F09162
:10090000FB010088F189E02D8CEF91E009958CEFD7
:1009100091E06EEA70E0C7DB8091BB00882319F09C
:100920008EEA90E0AADE909840D58091F401882369
:1009300019F01092F40147D575D58823B1F3909A38
:10094000E1D4E091FA01F091FB010484F585E02DFA
:100950000995DCD49098E091FA01F091FB010684AE
:10096000F785E02D0995882361F1909AE091FA01CD
:10097000F091FB010088F189E02D8CEF91E0099561
:100980008CEF91E06EEA70E08EDB84E092E06EEA3C
:1009900070E04AE151E013D48091F501882319F405
:1009A0006EEC71E002C06EEA71E08AE191E034DD44
:1009B0008091F50190E0882309F491E09093F5018E
:1009C00090988EEA90E020DFB0CF88E990E008951B
:1009D000009741F0DC01ECE7F1E088E001900D9236
:1009E0008150E1F7A4E8B1E0ECE7F1E088E00190A4
:1009F0000D928150E1F708958091AC009091AD0087
:100A0000892B31F01092AD001092AC0081E0089576
:100A10008CE791E064E871E048E050E072D5089519
:100A20000F931F93DF93CF93CDB7DEB7C850D1405C
:100A30000FB6F894DEBF0FBECDBF80E013D288ECB6
:100A400090E00197F1F7FE01399680E0EF93FF9374
:100A500000E810E41023C9F00000A39A0000000091
:100A60000000000000000000000000000000000086
:100A70000000000000000000A3983CE03A95F1F768
:100A800000000000069581F0E4CFA39A3FE03A957C
:100A9000F1F70000A3980000000000000000000033
:100AA0000000069509F0D5CFA39800E813E01023C5
:100AB000C9F00000A39A0000000000000000000040
:100AC0000000000000000000000000000000000026
:100AD0000000A3983CE03A95F1F70000000006956D
:100AE00081F0E4CFA39A3FE03A95F1F70000A39894
:100AF000000000000000000000000000069509F062
:100B0000D5CFA39800E8182F1023C9F00000A39AAE
:100B100000000000000000000000000000000000D5
:100B2000000000000000000000000000A3983CE06E
:100B30003A95F1F700000000069581F0E4CFA39A02
:100B40003FE03A95F1F70000A39800000000000094
:100B5000000000000000069509F0D5CFA398000022
:100B6000000000000000A39A000000000000000048
:100B70000000000000000000000000000000000075
:100B80000000000000000000A3980000000000002A
:100B90000000000000000000000013B31870E9F32B
:100BA00030E40FE30A9519F013B31870D9F78827CA
:100BB0008095FF91EF91C198EF93FF9388270027CD
:100BC0000395B1F09B99FCCF000008C00027039566
:100BD00079F09B99FCCF839551F001930027039501
:100BE00039F09B9BFCCF839511F00193EFCF000070
:100BF000FF91EF91813821F081E080938C0112C147
:100C0000DF01AE0147575F4F20E090818181981747
:100C100008F421E02D933296E417F507A9F7FE01B9
:100C2000319688E0DF011D928A95E9F74981FE013E
:100C3000799620E030E060E870E08081882339F028
:100C4000CB01022E02C0959587950A94E2F7482BB6
:100C50002F5F3F4F31962830310579F749834A811C
:100C6000FE01B19620E030E060E870E080818823EA
:100C700039F0CB01022E02C0959587950A94E2F7D0
:100C8000482B2F5F3F4F31962830310579F740953B
:100C90004A834B81FE01B99620E030E060E870E0C5
:100CA0008081882339F0CB01022E02C0959587956B
:100CB0000A94E2F7482B2F5F3F4F319628303105D9
:100CC00079F74B834C81FE01F19620E030E060E83B
:100CD00070E08081882311F080E007C0CB01022EF4
:100CE00002C0959587950A94E2F7482B2F5F3F4FF6
:100CF00031962830310569F74C834D81FE01F99614
:100D000020E030E060E870E08081882339F0CB019A
:100D1000022E02C0959587950A94E2F7482B2F5F23
:100D20003F4F31962830310579F740954D834E81FC
:100D3000FE01EF5BFF4F20E030E060E870E0808173
:100D4000882339F0CB01022E02C0959587950A942D
:100D5000E2F7482B2F5F3F4F31962830310579F766
:100D600040954E834F81FE013C9620E030E061E0EB
:100D700070E08081882339F0CB01022E02C0880FF9
:100D8000991F0A94E2F7482B2F5F3F4F3196253089
:100D9000310579F7FE01729620E030E060E270E004
:100DA0008081882339F0CB01022E02C0880F991F61
:100DB0000A94E2F7482B2F5F3F4F319623303105DD
:100DC00079F74F834885FE01759620E030E061E0B9
:100DD00070E08081882339F0CB01022E02C0880F99
:100DE000991F0A94E2F7482B2F5F3F4F319624302A
:100DF000310579F7898180937C018A8180937D0117
:100E00008B8180937E018C8180937F018D81809383
:100E100080018E81809381018F8180938201409334
:100E2000830180E0C85FDE4F0FB6F894DEBF0FBECF
:100E3000CDBFCF91DF911F910F91089510928C013A
:100E4000EFDD90E080918C01882309F491E0892FF7
:100E500008958FB7F894B99AC198A398AB988FBFAB
:100E6000DFDD08950F931F93DF93CF93CDB7DEB7E8
:100E7000C154D0400FB6F894DEBF0FBECDBFFE0107
:100E80003196EF93FF9300E8182F1023C9F000006C
:100E9000A39A000000000000000000000000000015
:100EA0000000000000000000000000000000A39807
:100EB0003CE03A95F1F700000000069581F0E4CFA0
:100EC000A39A3FE03A95F1F70000A39800000000D4
:100ED0000000000000000000069509F0D5CFA3989F
:100EE0000000000000000000000000000000000002
:100EF000A39A0000000000000000000000000000B5
:100F00000000000000000000000000000000A398A6
:100F100030E20FEF0A9529F113B31072D9F7C19897
:100F200000000000000000000000000000000000C1
:100F3000000000000000000000000000000023B3DB
:100F4000C19A287021933A9539F00FEF0A9549F02C
:100F500023B32870F1F6FACF882705C0C19A832FF2
:100F600002C088278095FF91EF91C1988F3F19F0BB
:100F700020E030E002C02FEF3FEFC901CF5BDF4F31
:100F80000FB6F894DEBF0FBECDBFCF91DF911F919A
:100F90000F9108951F921FB6EF93FF934F930F93F6
:100FA0001F937F93EDE8F1E001E20EC015E11A9581
:100FB000D9F040B34470D9F70000000000000000F1
:100FC000000000000000000034D0000040B300002A
:100FD000447041930A9539F015E11A9529F040B310
:100FE0004470D9F3E3CF04C041E2401B493049F0DB
:100FF0007F911F910F914F91FF91EF911FBE1F9015
:10100000189541E0E4EFF1E04083EDE8F1E015D020
:10101000442359F0413059F04F3F29F0909A000095
:1010200000009098E5CF34D0E3CF1FD0E1CF43D07C
:10103000DFCF12E01A95F1F708950F931F9344271D
:1010400000E81191112309F0402B0695D1F71F916B
:101050000F9108950F931F9300E8142F10231193FD
:101060000695D9F71F910F910895AF93BF93AEEEF8
:10107000B1E0EDE8F1E04D91EDDF4D91EBDF4D9109
:10108000E9DFBF91AF91EDE8F1E078E121D008957B
:10109000AF93BF93A1EFB1E0EDE8F1E04D91DADF5E
:1010A0004D91D8DF4D91D6DFBF91AF91EDE8F1E0E2
:1010B00078E10ED00895E5EFF1E07081772319F41F
:1010C000EEEAF1E002C0EEECF1E070E201D008954A
:1010D0003F934F937F9331913323E1F400008A9A39
:1010E0004FE04A95F1F700008A9842E04A95F1F7FF
:1010F0007A9589F700000000000000000000000061
:101100008A9A44E04A95F1F700008A987F914F91BE
:101110003F9108958A9A44E04A95F1F70000000053
:101120008A984CE04A95F1F7000000007A9599F60C
:101130000000000000000000000000008A9A44E067
:101140004A95F1F700008A987F914F913F91089559
:10115000FC0109C0992787FD90958617970711F420
:1011600041830895329680818F3FA1F70895FC0155
:101170008081823011F080E0089581810895FC0122
:101180008081833041F0843091F0813011F020E093
:1011900014C0218112C03281818137FF04C020E058
:1011A00038175CF009C020E083173CF005C020E050
:1011B0009181828189170CF021E0822F0895CF92CE
:1011C000DF92EF92FF920F931F93CF93DF938C01E7
:1011D0007B016A01FA0103C0838181833496808197
:1011E0008823D1F73DC0282F332727FD3095F801FC
:1011F0008181C82FDD27C7FDD095CC0FDD1FCC0F17
:10120000DD1FCC0DDD1D8881823081F08330D1F06F
:10121000813021F5220F331F220F331FC701820FA8
:10122000931FADDF9981982B998318C0F901EE0FB8
:10123000FF1FEE0FFF1FEE0DFF1D8081823071F446
:1012400081810BC0220F331F220F331FC701820F72
:10125000931F95DF882311F08A8189830E5F1F4FCA
:10126000F80180818F3F09F0BECFDF91CF911F91B0
:101270000F91FF90EF90DF90CF900895C198B99AA9
:101280000895892B11F41FBC089581E88FBD8AE071
:101290008EBD1BBC8FE18ABD08950F931F93CF9322
:1012A000DF93EC0100E911E081E090E0EADF80EB00
:1012B00094E0F8013197F1F70197D9F780E090E0D9
:1012C000E0DF84EF91E0F8013197F1F70197D9F76A
:1012D000219751F7DF91CF911F910F9108951F92A0
:1012E0000F920FB60F9211248F938091F6018C33D9
:1012F00018F48F5F8093F6018F910F900FBE0F90BF
:101300001F90189589B78E7F89BF089589B781602E
:1013100089BF089585E083BF12BE89B7816089BF08
:101320001092F60108958091F6018C3310F480E05C
:1013300008951092F60181E008958CE392E060E058
:1013400070E048E051E001D108958CE392E060E064
:1013500070E048E051E0E9D08CE392E06EE671E0A5
:1013600047E050E0CED0009719F420E030E01BC0F9
:10137000ACE3B2E0EEE6F1E087E001900D9281503F
:10138000E1F71092430284E492E06FEF70E040E0F6
:1013900051E0C4D08CE392E060E070E048E051E0BE
:1013A000D4D021E030E0C90108951FBC83E08EBD98
:1013B0001DBC1CBC1092F90186ED96E09093F801DB
:1013C0008093F701089508B602FE04C088B78460D0
:1013D00088BF1AC08CB59DB524E0833E9207D0F03B
:1013E00027E0813D920718F08E5E924002C086EDA4
:1013F00096E09093F8018093F7018091F701909126
:10140000F801825E944030F486ED96E09093F80106
:101410008093F7011DBC1CBC88B7846088BF109204
:10142000F90108958091F901882369F42CB53DB53F
:101430008091F7019091F8012817390720F081E099
:101440008093F901089580E00895629FD001739F11
:10145000F001829FE00DF11D649FE00DF11D929F50
:10146000F00D839FF00D749FF00D659FF00D99278F
:10147000729FB00DE11DF91F639FB00DE11DF91FB3
:10148000BD01CF011124089597FB092E05260ED02A
:1014900057FD04D014D00AD0001C38F45095409564
:1014A000309521953F4F4F4F5F4F0895F6F7909538
:1014B0008095709561957F4F8F4F9F4F0895A1E262
:1014C0001A2EAA1BBB1BFD010DC0AA1FBB1FEE1FBE
:1014D000FF1FA217B307E407F50720F0A21BB30B09
:1014E000E40BF50B661F771F881F991F1A9469F785
:1014F00060957095809590959B01AC01BD01CF01E1
:101500000895FB01DC0104C08D910190801921F444
:1015100041505040C8F7881B990B0895DC0101C069
:101520006D9341505040E0F70895DC01CB01FC0180
:10153000E199FECF06C0FFBBEEBBE09A31960DB23B
:101540000D9241505040B8F70895DC01CB0102C024
:101550002D9105D041505040D8F70895262FE1999C
:10156000FECF9FBB8EBB2DBB0FB6F894E29AE19ADB
:0A1570000FBE01960895F894FFCF16
:10157A000000010102020303040405050606070729
:10158A00080809090A0A0B0B0C0C0D0D0E0E0F0F99
:10159A001014111412141314141415141604170524
:1015AA00181419141A14FFFF0800000000000000A4
:1015BA00000029071005FC04E8041E0701000100C9
:1015CA00000001000000010000000100000001000D
:1015DA000000010000000300E000030020000300F7
:1015EA00E0000300200001000000010000000100EB
:1015FA0000000100000002000000020000000100DB
:10160A00000001000000030020000300E0000300C6
:10161A0020000300E0000400200004002000020073
:10162A0000000200000000000000010000000100AC
:10163A00000001000000010000000100000001009C
:10164A00000001000000010000000100000001008C
:10165A00000001000000010000000100000001007C
:10166A0000000200000002000000030081000300E5
:10167A007F000300810003007F0000000000474351
:08168A00324E363476310000C7
:00000001FF
